:100000000C942A000C9461010C9447000C94470056
:100010000C9447000C9447000C9447000C94470044
:100020000C9447000C9447000C9447000C94470034
:100030000C9447000C9490040C9447000C946804B2
:100040000C9447000C9447000C9447000C94470014
:100050000C94470011241FBECFE5D8E0DEBFCDBF12
:1000600012E0A0E6B0E0E8E5F9E302C005900D92E9
:10007000AE31B107D9F723E0AEE1B2E001C01D9285
:10008000AD3DB207E1F70E9409040C94AA1C0C9440
:10009000000087B3806B87BBBE98C49A83E58DB997
:1000A000709808958FB9779BFECF8FB10895809196
:1000B000BD039091BE03892B11F40E94DA14809144
:1000C0003F03813051F48091FF02811103C00E94EF
:1000D000AD0D38C00E94C01035C0823019F40E94A6
:1000E000EC1330C0833011F0803119F40E94B81243
:1000F00029C0843019F40E94B40F24C0853019F44B
:100100000E94560E1FC0863019F40E9419121AC0A0
:1001100099EF980F983018F40E940A0F13C08F308F
:1001200019F40E94CC0D0EC0813139F48091FF0288
:10013000882369F20E94221305C00E947C1581E089
:100140008093720280917202882321F00E94050937
:1001500010927202089585E083BF8FEF8ABB8FEB08
:1001600087BB80E284BB8AE781BB08958091A803A6
:10017000882319F081508093A8038091A7038823D6
:1001800019F081508093A70380916602882319F0AB
:100190008150809366028091D502882319F08150A6
:1001A0008093D5028091BD039091BE03009729F002
:1001B00001979093BE038093BD0380919902909123
:1001C0009A02883E2DEF920728F4019690939A02A6
:1001D000809399028091FE028F5F843119F08093A1
:1001E000FE020EC01092FE02809184029091850260
:1001F0008631910528F401969093850280938402BC
:1002000080913E038F5F883219F080933E030BC0CC
:1002100010923E038091FB029091FC020196909314
:10022000FC028093FB028091AD02882319F081507B
:100230008093AD02089510923F0310923F028FEF1A
:100240008093BF03109283021092AE028CE38093DE
:1002500066021092BE031092BD0310929A02109291
:1002600099021092440281E0809365021092FE028E
:1002700010923E031092FC021092FB021092B70201
:1002800010926A02109269021092880210928702FC
:100290001092AD021092FF02E1E4F3E0119283E0CC
:1002A000E934F807D9F708951092680210926702AE
:1002B0001092D5028BB780648BBF85B7836085BFF2
:1002C00008951F920F920FB60F9211248F939F9350
:1002D0008091D50281110EC0829B0CC08091670273
:1002E000909168020196909368028093670284E17E
:1002F0008093D5029F918F910F900FBE0F901F900A
:10030000189580918402909185028631910559F467
:1003100080917102806F8093710260E670E08CEAD8
:1003200093E00C94B919ECEAF3E08031910568F49C
:100330002CEB33E040E241932E173F07E1F7FC013D
:10034000E455FC4F2FEF208308958CEB93E02FEFC3
:1003500021938E179F07E1F708950E9481010E9463
:1003600076160C940509E6E3F3E080E09191913074
:1003700009F48F5F93E0EE33F907C1F70895809198
:100380004002811110C0A09141022AEFA29FC0013A
:1003900011249093280280932702B0E02AE33BE9DE
:1003A00042E250E029C0813099F4A091410224EF4B
:1003B00031E0A29FC001A39F900D112490932802C9
:1003C00080932702B0E024E736E345E450E014C010
:1003D0008230F1F4A09141022EEE32E0A29FC001E2
:1003E000A39F900D11249093280280932702B0E0E0
:1003F0002EEA31ED47E650E00E94AE1920E137E2E7
:1004000040E050E00E9476193093260220932502A6
:1004100008950F931F93CF93DF938AE08093400357
:100420008093CC0361E070E082E390E00E94BC1610
:1004300080914002882339F0813051F0C8EAD2E03F
:100440000EEE12E009C0C3EED0E00AEF10E004C0E7
:10045000C6ECD1E004EF11E08AE794E19093AC029E
:100460008093AB028DEA97E49093D7028093D602F3
:1004700083E393E3909364028093630284E1809327
:10048000CC038AE78093CD0362E070E08DE390E0D7
:100490000E94BC168091D6029091D7029093CC0313
:1004A0008093CD0362E070E080E490E00E94BC168F
:1004B00080916302909164029093CC038093CD036A
:1004C00062E070E087E490E00E94BC161092430264
:1004D000109242021092CC031092CD0362E070E0C1
:1004E00082E290E00E94BC161092DA021092D902C9
:1004F0001092CC031092CD0362E070E082E290E0B3
:100500000E94BC1620914102209FC001219F900DA6
:1005100011249093700280936F029093CC03809388
:10052000CD0362E070E08BE290E00E94BC16209167
:1005300041022C9FC0012D9F900D112490932E02FB
:1005400080932D029093CC038093CD0362E070E002
:100550008BE290E00E94BC168091AB029091AC02BD
:100560009093CC038093CD030FE212E0C0E0D0E083
:100570008091AB029091AC02F801819391938F012D
:1005800062E070E0CE01880F991F0E94BC16219690
:10059000C830D10569F78091D6029091D702909327
:1005A000CC038093CD0303E712E0C0E0D0E080915C
:1005B000D6029091D702F801819391938F01CE01D9
:1005C000880F991F62E070E041960E94BC16219648
:1005D000C830D10561F710926A0210926902109238
:1005E00088021092870210928302DF91CF911F91AF
:1005F0000F910C94BF01FF920F931F93CF93DF9342
:10060000C82F1092CC031092FD0261E070E08EE2E0
:1006100090E00E94BC16C093CC03C093D40261E06A
:1006200070E080E390E00E94BC1681E08093CC03F0
:100630008093400261E070E085E490E00E94BC1687
:1006400084E0809341028093CC0361E070E083E416
:1006500090E00E94BC1606E313E0C0E0D0E0FF2467
:10066000F394F801C430D10514F4F08201C0108273
:10067000F80181918F018093CC0361E070E0CE019D
:10068000C4960E94BC162196C830D10551F7DF915F
:10069000CF911F910F91FF900C9409028091D40289
:1006A0000C94FB020F931F93CF93DF9382E390E0B0
:1006B0000E94A016809340038B3038F080E0DF91D9
:1006C000CF911F910F910C94FB020FE212E0C0E05A
:1006D000D0E0CE01880F991F0E94A716F8018193E0
:1006E00091938F012196C830D10599F703E712E065
:1006F000C0E0D0E0CE01880F991F41960E94A71656
:10070000F801819391938F012196C830D10591F71B
:1007100006E313E0C4E3D0E0CE010E94A016F80186
:1007200081938F012196CC33D105B1F782E290E01D
:100730000E94A716909343028093420285E290E0C4
:100740000E94A7169093700280936F0288E290E057
:100750000E94A7169093DA028093D9028BE290E070
:100760000E94A71690932E0280932D028DE390E0B5
:100770000E94A7169093AC028093AB0280E490E0B5
:100780000E94A7169093D7028093D60287E490E048
:100790000E94A71690936402809363028EE290E019
:1007A0000E94A0168093FD0280E390E00E94A016B4
:1007B0008093D40285E490E00E94A01680934002CA
:1007C00083E490E00E94A01680934102DF91CF91D4
:1007D0001F910F910C94BF011BBA18BA15BA12BA27
:1007E000C49AAD9A0E94AB00C49AAD9A0E940316B7
:1007F0000E94DB080E9454010E9453040E94490099
:10080000789489E190E00E9433160E941B010C94B9
:1008100052030E94EC03109235031092340310929D
:100820002C0210922B021092D3021092D2029EE060
:1008300088E10FB6F894A89581BD0FBE91BDC6EAB8
:10084000C2BF88B7816088BFA8950E9448162091D2
:10085000990230919A0280913F022830324040F450
:10086000813019F40E94AD0107C00E94110904C033
:100870008130C1F30E9457000E94C9060E948A0875
:100880008091990290919A028935924010F00E94CD
:100890003F170E946B160E94B6000E94B20408B671
:1008A00000FEFDCFCDCF1092A60381E08093AA0376
:1008B0001092A5031092A8031092A9031092A70307
:1008C00086E080BD10BC87E189B988E98AB90895BE
:1008D0001F920F920FB60F9211248F93EF93FF93F5
:1008E000E091AA038091A503E81758F4F0E0E65BD5
:1008F000FC4F80818CB98091AA038F5F8093AA03FB
:1009000007C01092A5031092AA03939888E98AB9A8
:10091000FF91EF918F910F900FBE0F901F90189540
:100920001F920F920FB60F9211248F939F93EF9304
:10093000FF939CB184E08093A7038091A903E82FE3
:10094000F0E0E556FC4F90838A3018F48F5F809377
:10095000A903FF91EF919F918F910F900FBE0F9080
:100960001F9018958091A6038823A1F08091A80379
:10097000811110C01092A6035E9A81E08093AA03B1
:10098000939A88E58AB981E090E00E9433168091BD
:100990004A038CB908958091D8028F5F09F48EE1E3
:1009A0008093D80286E080934A038091D40280939A
:1009B0004B038091FD02811115C090915902209145
:1009C0005A0220934C0390934D0390914202209140
:1009D000430220934E0390934F0390916F02209116
:1009E000700214C09091290220912A0220934C0396
:1009F00090934D039091D9022091DA0220934E03F7
:100A000090934F0390912D0220912E02209350033A
:100A1000909351039091D802909352039091400388
:100A2000909353039091670220916802209354039E
:100A3000909355031092560397ED9093570390911E
:100A40009B0220919C02209358039093590390910C
:100A50009D0220919E0220935A0390935B039091F4
:100A60009F022091A00220935C0390935D039091DC
:100A7000A1022091A20220935E0390935F039091C4
:100A8000A3022091A40220936003909361039091AC
:100A9000A5022091A6022093620390936303909194
:100AA000A7022091A802209364039093650390917C
:100AB000A9022091AA022093660390936703909164
:100AC000AB022091AC02209368039093690390914C
:100AD000D6022091D70220936A0390936B039091E2
:100AE00063022091640220936C0390936D03811143
:100AF00005C09091690220916A0204C0909187021A
:100B00002091880220936E0390936F03909141028D
:100B100090937003909140029093710380937203BD
:100B2000E1E4F3E029E433E080E0869591919111CE
:100B300080682E173F07C9F78093730310927403E0
:100B400010927503109276031092770380912F0212
:100B500090913002909378038093790380913102D1
:100B60009091320290937A0380937B0380913302B9
:100B70009091340290937C0380937D0380913502A1
:100B80009091360290937E0380937F038091370289
:100B90009091380290938003809381038091390271
:100BA00090913A02909382038093830380913B0259
:100BB00090913C02909384038093850380913D0241
:100BC00090913E02909386038093870380917302F5
:100BD00090917402909388038093890380917502A9
:100BE0009091760290938A0380938B038091770291
:100BF0009091780290938C0380938D038091790279
:100C000090917A0290938E0380938F0380917B0260
:100C100090917C02909390038093910380917D0248
:100C200090917E02909392038093930380917F0230
:100C30009091800290939403809395038091810218
:100C4000909182029093960380939703E6E3F3E0FA
:100C50002EE333E080E086959191911180682E1704
:100C60003F07C9F780939803EAE4F3E029E933E00A
:100C700080E090E04191840F911D2E173F07D1F73E
:100C80009093990380939A031092AA0381E580932D
:100C9000A50382E08093A80381E08093A6030895D2
:100CA00081E080934A0380934B0390919B02809153
:100CB0009C0290934C0380934D0390919D028091F0
:100CC0009E0290934E0380934F0390919F028091D8
:100CD000A00290935003809351039091A1028091C0
:100CE000A20290935203809353039091A3028091A8
:100CF000A40290935403809355039091A502809190
:100D0000A60290935603809357039091A702809177
:100D1000A80290935803809359039091A90280915F
:100D2000AA0290935A0380935B038091670290918B
:100D3000680290935C0380935D03809171028093BD
:100D40005E0380935F03EAE4F3E080E090E02191AA
:100D5000820F911D23E0E036F207C9F790936003FC
:100D6000809361031092AA0388E18093A50384E035
:100D70008093A80381E08093A6030895282FFC01A7
:100D800080E09E2F921B961718F49191890FF9CF4E
:100D90000895EF92FF921F93CF93DF938091A70363
:100DA00081112FC18091A903882309F42AC12091C0
:100DB0009B03243509F58330E1F480919C0383354E
:100DC00081F480919D038435A1F481E080933F02FA
:100DD0001092850210928402109271020E945401B6
:100DE00006C0813031F480919D03853511F40E9455
:100DF00050061092A90305C14091990250919A02A0
:100E0000403D5240B0F390919C03223561F4209113
:100E1000D4029213EECF833061F7C0919D0362E05C
:100E20008BE993E0E9C0233509F0D5C0863008F49A
:100E3000D2C08091D4029813DCCFC0919E036FEF93
:100E40006C0F8BE993E00E94BE06EC2FF0E0E656B3
:100E5000FC4F90819813CDCF80919D0381111AC0D2
:100E600010919F0376E3E72E73E0F72EC4E3D0E002
:100E7000812F8170F70181937F0116958093CC03B8
:100E800061E070E0CE010E94BC162196CC33D10502
:100E900079F79EC0813059F520919F0330E0322FC1
:100EA00022278091A003280F311D8091FD0281111E
:100EB0000DC080916F029091700296958795821770
:100EC000930708F485C0A4E1B0E00CC080912D0226
:100ED00090912E02969587958217930708F478C013
:100EE000AAE0B0E00E9498190E94480C71C08230BC
:100EF00019F40E94880B6CC08330B9F420919F03D1
:100F000030E0322F22278091A003280F311D8091DD
:100F1000FD02811103C0A4E1B0E002C0AAE0B0E08C
:100F20000E9498190E944F0953C08430D1F48091D7
:100F30009F0390914003913009F44AC09DEF980FB0
:100F4000963008F045C090914102891709F440C0DD
:100F5000809341028093CC0361E070E083E490E0F1
:100F60002DC0853099F480919F03823088F590914F
:100F7000FD02891769F18093FD028093CC0361E043
:100F800070E08EE290E00E94BC1622C08630D9F458
:100F900080919F03909140039130D1F09FEF980F83
:100FA0009230B0F490914002891791F08093400202
:100FB0008093CC0361E070E085E490E00E94BC1671
:100FC0000E94090205C0873009F013CF0E944E032A
:100FD0000E94CB040ECF923509F00BCF20919D03D8
:100FE0009091D402291305CF843009F002CFC0912B
:100FF0009E0362E08CE993E00E94BE06C813F9CE1E
:10100000E7CFDF91CF911F91FF90EF9008950000FF
:1010100000000000000000000000000000000000D0
:1010200000000000000000000000000000000000C0
:1010300000000000000000000000000000000000B0
:1010400000000000000000000000000000000000A0
:101050000000000000000000000000000000000090
:1010600000000000000000000000000000000895E3
:10107000CF93C4980E940708C6B3C49A0E94070879
:10108000C6FBCC27C0F981E08C27CF910895CF9380
:10109000C82FC4980E9407088C2F8F70806A0E9406
:1010A000520080E00E94520080E00E945200C49AE8
:1010B000CF910C940708CF92DF92EF92FF92CF93DB
:1010C000C82FC4980E9407088C2F8F70806A0E94D6
:1010D0005200C82ED12CE12CF12C7601DD24CC2439
:1010E00080E00E945200D82A80E00E945200C82A64
:1010F000C49A0E940708D701C60125E0B695A795B6
:10110000979587952A95D1F7CF91FF90EF90DF9033
:10111000CF9008950F931F93CF93DF930E943808C9
:10112000882309F443C0C0912203D0E08E010F5FF1
:101130001F4F07701127802F0E945B08CC0FDD1F07
:10114000C556DD4F998388838091220390E0FC018E
:10115000EA5CFC4F2081DC01AF5BBC4F222361F0D5
:10116000880F991FFC01E556FD4F808191818E51BA
:1011700095408A329C45B8F41C9200932203E6E322
:10118000F3E0A1E4B3E080E09191992321F09C91F8
:10119000911101C08F5F119693E0EE33F907A1F72B
:1011A0008093FF0203C081E08C93E7CFDF91CF9162
:1011B0001F910F9108950E94490080E00C94470808
:1011C0000F931F93CF93DF93D82FC92F80E00E94F6
:1011D000BE150D2F1C2FD0E0F801C1918F01CC233B
:1011E00079F0D13169F0D83019F488E00E94BE1549
:1011F000CA3008F4C05D8C2F0E94D615DF5FECCF9B
:10120000DF91CF911F910F9108950E94D3158CEA21
:1012100093E00E94E0088091440281110C94C8156B
:1012200008958091990290919A020097F1F41F928B
:101230008FE08F931F9282E08F9381E790E09F93DE
:101240008F938CEA93E09F938F930E94C01980E163
:101250008093BF03109244028DB79EB708960FB6D5
:10126000F8949EBF0FBE8DBF09C0883C910541F424
:1012700065E870E08CEA93E00E94B9190C940509C6
:10128000883621E0920719F466E970E0F3CF8956B9
:1012900091408F39910510F40C948A0808952F928B
:1012A0003F925F926F927F928F929F92AF92BF9286
:1012B000CF92DF92EF92FF920F931F93CF93DF9322
:1012C000CDB7DEB728970FB6F894DEBF0FBECDBFFF
:1012D0003B018C839B8326E333E03A832983FBE93C
:1012E000CF2EF2E0DF2EA1E48A2EA3E09A2ED401C5
:1012F000960116E3A12E13E0B12E60E070E0CB0161
:10130000E12CF12CF50141915F01442369F0F901D1
:10131000408151811C91111107C0640F751F811DFF
:10132000911DFFEFEF1AFF0A2E5F3F4F11964EE31C
:10133000A41643E0B40631F7E114F10409F45BC1EB
:101340005701B694A7946A0D7B1D811D911D8701DD
:1013500020E030E0A90198010E947619522E222E39
:10136000332E8091AB029091AC028101081B190BC6
:101370008091FD02B301882329F08C819B810E941A
:10138000D51602C08C819B819B01AC016AE0220FC3
:10139000331F441F551F6A95D1F7C801969587954D
:1013A000280F391F411D511DCA01B901980140E0A4
:1013B00050E00E947619C501820F931FB7010E9469
:1013C000621980914002811107C0685371406E39E3
:1013D000710508F012C108C0813071F46157724084
:1013E0006933714008F009C183E7A82E82E0B82E66
:1013F00091E1E92EF12C2CC08230B1F76A5A73408A
:10140000653D714008F0F9C0EFCFF6018081918110
:10141000F4012081213019F1F50180839183F2E0FC
:10142000AF0EB11C9093CC038093CD0362E070E0CB
:10143000C7010E94BC1622E0E20EF11C32E0C30E8E
:10144000D11C4FEF841A940A51E2E516F10451F0D1
:10145000E981FA818191FA83E9838111D6CF80E015
:1014600090E0DACF3092D7022092D6023092CC03AD
:101470005092CD0362E070E080E490E00E94BC16E0
:1014800000936302109364021093CC030093CD0386
:1014900062E070E087E490E00E94BC168091FD025B
:1014A000811116C06092CD027092CE028C81809321
:1014B000CF029B819093D002B3010E94E916609302
:1014C000B9027093BA028093BB029093BC0216C01B
:1014D0006092B9027092BA02EC81E093BB02FB8188
:1014E000F093BC02B301CF010E94D5166093CD02E8
:1014F0007093CE028093CF029093D0028091CD0260
:101500009091CE02A091CF02B091D002BC01CD014A
:10151000665F7F4F8F4F9F4F24E130E040E050E007
:101520000E947619CA01B9013093700220936F02AC
:1015300030935A0220935902209142023091430283
:10154000260F371F309309032093080344E050E02F
:1015500081E292E00E9403178091B9029091BA0251
:10156000A091BB02B091BC02BC01CD016B5F7F4F6B
:101570008F4F9F4F2AE030E040E050E00E94761904
:10158000CA01B90130932E0220932D0230932A0212
:10159000209329022091D9023091DA02260F371FB9
:1015A000309346022093450244E050E08BE692E0FF
:1015B0000E94031780916F02909170029093CC0368
:1015C0008093CD0362E070E085E290E00E94BC165B
:1015D00080912D0290912E029093CC038093CD03A5
:1015E00062E070E08BE290E00E94BC1682E08093A3
:1015F000650280E003C083E001C084E028960FB656
:10160000F894DEBF0FBECDBFDF91CF911F910F9138
:10161000FF90EF90DF90CF90BF90AF909F908F9012
:101620007F906F905F903F902F900895809140033E
:10163000813069F5E6E3F3E0A1E4B3E080E090E017
:101640002191222321F02C91213009F0019611964D
:1016500023E0EE33F207A1F7892BD9F0409147023E
:101660005091480260E070E08BE0440F551F661F08
:10167000771F8A95D1F74756564E6F4F7F4F81E0BF
:101680004A3053436942710528F080E0089582E0B2
:10169000089583E008958091AB029091AC029093FD
:1016A000CC038093CD0362E070E08DE390E00E9474
:1016B000BC1680914202909143029093CC03809398
:1016C000CD0362E070E082E290E00E94BC1680915F
:1016D000D9029091DA029093CC038093CD0362E01B
:1016E00070E088E290E00E94BC1680914003813057
:1016F00059F081E0809340038093CC0361E070E077
:1017000082E390E00E94BC1681E080936502089518
:101710006F927F928F929F92AF92BF92CF92DF9201
:10172000EF92FF920F931F93CF93DF9336E3832EB5
:1017300033E0932E4FE2642E42E0742E5BE9A52E37
:1017400052E0B52E61E4C62E63E0D62E00E010E034
:10175000C0E0D0E0E12CF12CF40181914F0188230D
:1017600059F0F50180819181F6012081211104C099
:10177000080F191F219602C080E090E0F3018193C9
:1017800091933F019093CC038093CD0362E070E08E
:10179000C7010E94BC16F2E0EF0EF11C82E0A80E19
:1017A000B11CEFEFCE1ADE0AF0E1EF16F104A1F65C
:1017B000209709F45EC0CE0196958795800F911F02
:1017C000BE010E9462197093AC026093AB028091DB
:1017D0000803909109039093430280934202809101
:1017E0004502909146029093DA028093D9021092BA
:1017F0005A021092590210922A0210922902109253
:10180000CD021092CE021092CF021092D00210920E
:10181000B9021092BA021092BB021092BC0210924E
:101820006A0210926902109288021092870244E0C4
:1018300050E060E070E081E292E00E940317609166
:10184000290270912A0244E050E08BE692E00E9467
:101850000317DF91CF911F910F91FF90EF90DF90D1
:10186000CF90BF90AF909F908F907F906F900C948F
:101870004B0BDF91CF911F910F91FF90EF90DF9075
:10188000CF90BF90AF909F908F907F906F90089572
:101890008F929F92AF92BF92CF92DF92EF92FF9280
:1018A0000F931F93CF93DF934B015C018091FD0257
:1018B000811130C0C0904202D0904302C501B401F2
:1018C000665F7F4F8F4F9F4F24E130E040E050E054
:1018D0000E947619E9013093430220934202E0907E
:1018E0006F02F09070020091080310910903C50186
:1018F000B4010E94E9166B5F7F4F8F4F9F4F2AE024
:1019000030E040E050E00E9476193093DA022093F4
:10191000D9022FC0C090D902D090DA02C501B4011B
:101920006B5F7F4F8F4F9F4F2AE030E040E050E0E9
:101930000E947619E9013093DA022093D902E090EF
:101940002D02F0902E020091450210914602C50131
:10195000B4010E94D516665F7F4F8F4F9F4F24E1E1
:1019600030E040E050E00E9476193093430220932B
:101970004202A0916302B0916402A7015695479577
:101980004701A12CB12CE090AB02F090AC02CC1539
:10199000DD05A0F09E012C193D090E94A719640FD6
:1019A000751F811D911DA50194010E947619DA0110
:1019B000C9018E0D9F1DA11DB11D14C096012C1BC8
:1019C0003D0B0E94A719640F751F811D911DA50174
:1019D00094010E947619C701A0E0B0E0821B930B2E
:1019E000A40BB50B9093AC028093AB0240914202E2
:1019F0005091430260910803709109038091D902CC
:101A00009091DA022091450230914602C017D10729
:101A1000A8F4641B750B70935A02609359021092DC
:101A20006A0210926902281B390B30932A02209314
:101A30002902109288021092870214C010925A0252
:101A400010925902461B570B50936A024093690249
:101A500010922A0210922902821B930B9093880203
:101A600080938702E0915902F0915A029F01A4E10C
:101A7000B0E00E9498196093CD027093CE028093DB
:101A8000CF029093D0022091290230912A02AAE03D
:101A9000B0E00E9498196093B9027093BA028093E3
:101AA000BB029093BC0244E050E0BF0181E292E0AF
:101AB0000E9403176091290270912A0244E050E0CD
:101AC0008BE692E00E940317DF91CF911F910F9157
:101AD000FF90EF90DF90CF90BF90AF909F908F904E
:101AE0000C944B0B80913F03813149F48091FD02AE
:101AF000813061F488EC9FEAA0E0B0E00BC0833055
:101B000029F482E390E0A0E0B0E004C08FE996E819
:101B1000A1E0B0E08093C0039093C103A093C203FF
:101B2000B093C30308956093C5037093C603809375
:101B3000C7039093C8030E94720D81E080937202E4
:101B40000895809140038A3011F485E001C081E05E
:101B500080933F031092D102089580913F039FEF3D
:101B6000980F9E3010F48F5F12C08F3031F4809147
:101B70008602813031F480E10AC090EF980F9230F4
:101B800018F410923F0305C0811103C081E18093D6
:101B90003F031092D10208958091D102811112C0A9
:101BA0006091FD0270E080E090E00E94930D85E07E
:101BB0008093AB038FE08093BF038091D1028F5F4E
:101BC0008093D10281E00E946E16811111C088E0DD
:101BD0000E946E16882371F08091C5038093FD02E8
:101BE0008093CC0361E070E08EE290E00E94BC162E
:101BF0000C94AD0D84E00E946E168823C9F080918C
:101C0000C5039091C603A091C703B091C803892B67
:101C10008A2B8B2B99F481E090E0A0E0B0E08093D8
:101C2000C5039093C603A093C703B093C8030EC027
:101C300082E00E946E168111E2CF0BC01092C503A4
:101C40001092C6031092C7031092C80381E08093DC
:101C5000720267EA70E08CEA93E00E94B919809101
:101C6000C5039091C603A091C703B091C803009724
:101C7000A105B10541F48CE68093B90382E6809317
:101C8000BA0383E710C00197A105B10529F48BE6DB
:101C90008093BA0387E607C08EE68093B9038FE28C
:101CA0008093BA0381E68093BB030895CF9380911C
:101CB000D102811125C06091400270E080E090E087
:101CC0000E94930DC1E0C093AB038FE08093BF03EC
:101CD0008091D1028F5F8093D102809140038A303E
:101CE00069F4109240031092CC0361E070E082E34B
:101CF00090E00E94BC16C093860202C01092860239
:101D000081E00E946E16882319F0CF910C94AD0DDE
:101D100088E00E946E168823B9F08091C5039091E7
:101D20004002891791F390914003913071F38093B1
:101D300040028093CC0361E070E085E490E00E9473
:101D4000BC160E940902E1CF80914003813079F1F5
:101D500082E00E946E16882389F08091C5039091DD
:101D6000C603A091C703B091C8030197A105B105AF
:101D700059F482E090E0A0E0B0E00AC084E00E9464
:101D80006E168111EACF0FC081E090E0A0E0B0E0D4
:101D90008093C5039093C603A093C703B093C80371
:101DA00081E08093720281E08093440202C010922D
:101DB000440268EB70E08CEA93E00E94B9198091CC
:101DC000C5039091C603A091C703B091C8030097C3
:101DD000A105B10511F484E30FC081309105A1057F
:101DE000B10511F488E308C00297A105B10539F4E3
:101DF00081E38093B90382E38093BA0309C08EE63E
:101E00008093B9038FE28093BA0381E68093BB038A
:101E1000CF9108958091D102811121C0E0913F03BB
:101E2000E750E093B802F0E0EA5CFC4F608170E0BC
:101E300080E090E00E94930D85E08093AB038FE0FB
:101E40008093BF038091D1028F5F8093D102E09194
:101E5000B802F0E0EA5CFC4F80818093200281E0D0
:101E60000E946E16811115C088E00E946E168823AC
:101E700091F08091B80290E02091C503FC01EA5CEA
:101E8000FC4F20832093CC0361E070E0C4960E9455
:101E9000BC160C94AD0D84E00E946E16882339F0B8
:101EA0000E94B30190914102891738F40AC082E080
:101EB0000E946E168111F4CF22C0809120028130E1
:101EC00099F48091C5039091C603A091C703B09186
:101ED000C80321E082278093C5039093C603A09393
:101EE000C703B093C80308C01092C5031092C6037D
:101EF0001092C7031092C80381E08093720281E0C0
:101F00008093440269EC70E08CEA93E00E94B91976
:101F10008091B8028F5C8093AF038091C50390914C
:101F2000C603A091C703B091C8030097A105B105EE
:101F300029F48EE48093BA038FE613C00197A105BC
:101F4000B10541F489E58093B90385E68093BA032E
:101F500083E707C08EE68093B9038FE28093BA03CC
:101F600081E68093BB0308958091D102811110C056
:101F700060E070E0CB010E94930D85E08093AB039D
:101F80008FE08093BF038091D1028F5F8093D10255
:101F900081E00E946E1681110C94AD0D88E00E94C4
:101FA0006E16882339F08091C5038823A9F30E9417
:101FB0004E03F2CF84E00E946E168823C9F0809110
:101FC000C5039091C603A091C703B091C803892BA4
:101FD0008A2B8B2B99F481E090E0A0E0B0E0809315
:101FE000C5039093C603A093C703B093C8030EC064
:101FF00082E00E946E168111E2CF0BC01092C503E1
:102000001092C6031092C7031092C80381E0809318
:10201000720281E0809344026AED70E08CEA93E002
:102020000E94B9198091C5039091C603A091C7037E
:10203000B091C8030097A105B10529F48EE48093FF
:10204000BA038FE613C00197A105B10541F489E5F4
:102050008093B90385E68093BA0383E707C08EE6D1
:102060008093B9038FE28093BA0381E68093BB0328
:1020700008958091AB03813059F0823071F0833044
:1020800089F08430A1F061E070E080E090E0089594
:1020900060E177E280E090E0089568EE73E080E030
:1020A00090E0089564E670E080E090E008956AE0D2
:1020B00070E080E090E008958F929F92AF92BF927F
:1020C000CF92DF92EF92FF928091AB038F5F80936C
:1020D000AB038091BF038F5F8093BF038090C503E4
:1020E0009090C603A090C703B090C8038091C0032E
:1020F0009091C103A091C203B091C30388159905C3
:10210000AA05BB05E0F40E9439109B01AC01AAE0CE
:10211000B0E00E94AE196B017C01C501B401A701BA
:1021200096010E947619C701B6010E945219609368
:10213000C5037093C6038093C7039093C8030E949E
:1021400039109B01AC016091C5037091C603809169
:10215000C7039091C8030E947619CA01B9012AE009
:1021600030E040E050E00E9476196093C403FF9095
:10217000EF90DF90CF90BF90AF909F908F90089599
:10218000CF938091D102811110C060E070E0CB014B
:102190000E94930D81E08093AB038BE08093BF039B
:1021A0008091D1028F5F8093D102C1E0C09344023D
:1021B0008091C8038F938091C7038F938091C6034A
:1021C0008F938091C5038F938BEE90E09F938F93B5
:1021D0008CEA93E09F938F930E94C01981E00E9444
:1021E0006E162DB73EB7285F3F4F0FB6F8943EBF2F
:1021F0000FBE2DBF882319F0CF910C94AD0D88E050
:102200000E946E168823A1F08091AB03853039F4CB
:102210000E94880B10923F031092D10209C0809156
:10222000D1028F5F8093D1020E945C10C093720232
:10223000CF9108958F929F92AF92BF92CF92DF92EB
:10224000EF92FF920F931F93CF930E9439104B018F
:102250005C01C090C503D090C603E090C703F09026
:10226000C803C091C403C93068F5C701B601A50110
:1022700094010E947619C501B4010E945219DC0133
:10228000CB01880D991DAA1DBB1D0091C0031091A3
:10229000C1032091C2033091C303081719072A070D
:1022A0003B0780F0C80CD91CEA1CFB1CC092C5037C
:1022B000D092C603E092C703F092C803CF5FC093E9
:1022C000C40314C0AC2FB0E0A50194010E94AE1964
:1022D000C61AD70AE80AF90AC092C503D092C60303
:1022E000E092C703F092C8031092C40381E0809388
:1022F0007202CF911F910F91FF90EF90DF90CF90DE
:10230000BF90AF909F908F9008954F925F926F9281
:102310007F928F929F92AF92BF92CF92DF92EF9275
:10232000FF92CF93DF9300D000D0CDB7DEB70E94ED
:1023300039106B017C012091C4036091C503709139
:10234000C6038091C7039091C803222391F0DC015A
:10235000CB018C199D09AE09BF098093C5039093E9
:10236000C603A093C703B093C80321502093C403AE
:102370004AC0A70196010E9476194B015C01C70172
:10238000B6010E94521969837A838B839C83609182
:10239000C0037091C1038091C2039091C303A70150
:1023A00096010E947619C701B6010E9452192B01AD
:1023B0003C01E9E0AE2FB0E0A70196010E94AE1902
:1023C00029813A814B815C81260F371F481F591F95
:1023D000DA01C9012FEF2E0F481659066A067B064F
:1023E00010F4E22FE7CFE093C403AA24BB24880DA6
:1023F000991DAA1DBB1D8093C5039093C603A0938E
:10240000C703B093C80381E0809372020F900F90CE
:102410000F900F90DF91CF91FF90EF90DF90CF90D2
:10242000BF90AF909F908F907F906F905F904F90F4
:1024300008958091D102811122C080914102835080
:10244000863058F084E0809341028093CC0361E0B1
:1024500070E083E490E00E94BC166091410270E05D
:1024600080E090E00E94930D84E08093AB038EE0C7
:102470008093BF030E945C1081E08093D10281E0D1
:102480000E946E1681110C94AD0D88E00E946E16AC
:10249000882399F08091C50390914102891799F39F
:1024A000809341028093CC0361E070E083E490E08C
:1024B0000E94BC160E940902E6CF80914003813041
:1024C000B1F182E00E946E168823D1F00E94B30120
:1024D0004091C5035091C6036091C7037091C80332
:1024E00090E0A0E0B0E084179507A607B707D8F4FE
:1024F0004330510561057105B0F00E94851113C08C
:1025000084E00E946E16882371F08091C50390913B
:10251000C603A091C703B091C8030897A105B105F0
:1025200010F40E941A1181E08093440202C01092BC
:1025300044028091C8038F938091C7038F93809149
:10254000C6038F938091C5038F938CEF90E09F9388
:102550008F938CEA93E09F938F930E94C0198DB75D
:102560009EB708960FB6F8949EBF0FBE8DBF089514
:102570008091D102811112C06091D40270E080E09C
:1025800090E00E94930D83E08093AB038DE08093F5
:10259000BF030E945C1081E08093D10281E00E9421
:1025A0006E1681110C94AD0D88E00E946E16882382
:1025B000D9F08091D102823079F48091C503809363
:1025C000D4028093CC0361E070E080E390E00E944D
:1025D000BC1610923F0308958F5F8093D1020E9432
:1025E0005C1081E08093720282E00E946E1681117D
:1025F0000E94851184E00E946E1681110E941A11BA
:1026000081E0809344028091C8038F938091C70337
:102610008F938091C6038F938091C5038F9381E13F
:1026200091E09F938F938CEA93E09F938F930E9406
:10263000C0198DB79EB708960FB6F8949EBF0FBE0F
:102640008DBF08958091D102863010F01092D10292
:102650008091D102811127C00E94160B80931F0226
:102660008091FD02811109C06091CD027091CE026E
:102670008091CF029091D00208C06091B902709110
:10268000BA028091BB029091BC020E94930D1092FD
:10269000AB038AE08093BF030E945C108091D1025B
:1026A0008F5F8093D10281E00E946E1681110C949D
:1026B000AD0D80911F02811172C088E00E946E16DC
:1026C000882311F18091AB03853099F46091C503A3
:1026D0007091C6038091C7039091C8030E944F096F
:1026E00080931F02811177C010923F031092D10294
:1026F00008958091D1028F5F8093D1020E945C1077
:1027000081E0809372020EC084E00E946E168823DE
:1027100019F00E941A1106C082E00E946E16811103
:102720000E94851181E0809344024091FD02309126
:10273000C8032091C7039091C6038091C50341113E
:1027400017C03F932F939F938F9382E291E09F93C3
:102750008F938CEA93E09F938F930E94C0198DB75B
:102760009EB708960FB6F8949EBF0FBE8DBF089512
:102770003F932F939F938F9383E391E09F938F9346
:102780008CEA93E09F938F930E94C0198DB79EB7F8
:1027900008960FB6F8949EBF0FBE8DBF0895109295
:1027A000440291E090937202823019F464E471E083
:1027B0000EC0833019F465E571E009C0813019F469
:1027C00066E671E004C0843031F467E771E08CEABA
:1027D00093E00C94B9190895CF92DF92EF92FF9293
:1027E0008091D10281111DC010921E0220914202DF
:1027F00030914302A4E1B0E00E9498192091FD02BB
:10280000213011F40E94E9160E94930D81E080931B
:10281000AB038BE08093BF038091D1028F5F8093E5
:10282000D10281E00E946E16882331F0FF90EF9074
:10283000DF90CF900C94AD0D88E00E946E16882337
:1028400009F44FC08091AB03853009F03FC08091FF
:10285000FD02C090C503D090C603E090C703F0907E
:10286000C803811119C0C701B601665F7F4F8F4F42
:102870009F4F24E130E040E050E00E9476198091C3
:102880006F02909170029695879582179307A8F42E
:1028900081E080931E0289C0C701B6016B5F7F4F44
:1028A0008F4F9F4F2AE030E040E050E00E947619C1
:1028B00080912D0290912E02E6CFC701B6010E94B1
:1028C000480C10923F031092D1026FC08091D10248
:1028D0008F5F8093D1020E945C1081E0809372022E
:1028E00017C084E00E946E16882339F080911E0282
:1028F000811103C00E941A110BC082E00E946E1663
:10290000882331F080911E02811102C00E9485113E
:1029100080911E0281113DC081E08093440240916C
:10292000FD023091C8032091C7039091C6038091A6
:10293000C503411117C03F932F939F938F9388E84E
:1029400091E09F938F938CEA93E09F938F930E94E3
:10295000C0198DB79EB708960FB6F8949EBF0FBEEC
:102960008DBF23C03F932F939F938F9389E991E06D
:102970009F938F938CEA93E09F938F930E94C0194B
:102980008DB79EB708960FB6F8949EBF0FBE8DBF49
:102990000CC0813051F46AEA71E08CEA93E0FF9058
:1029A000EF90DF90CF900C94B919FF90EF90DF90EB
:1029B000CF90089510923F0308959091AE028091B8
:1029C0006602811109C081E0890F8C3018F4809370
:1029D000AE0202C01092AE028091AE02883060F565
:1029E00021E0280FE82FF0E0EF5BFC4F3081313021
:1029F00011F0822FF3CF8093AE02981709F479C0BB
:102A00009CE390936602109244028830D8F490E0E0
:102A100001969F938F938BEB91E09F938F938CEA1A
:102A200093E09F938F930E94C0190F900F900F9087
:102A30000F900F900F9008958093AE029813E0CFFF
:102A400010924402883039F480914003811103C010
:102A50006DEC71E008C08091690290916A0249971B
:102A600030F06EED71E08CEA93E00C94B91980912E
:102A7000FD0281111FC08091D0028F938091CF02FF
:102A80008F938091CE028F938091CD028F938FEEA2
:102A900091E09F938F938CEA93E09F938F930E9492
:102AA000C0198DB79EB708960FB6F8949EBF0FBE9B
:102AB0008DBF08958091BC028F938091BB028F934C
:102AC0008091BA028F938091B9028F9380E092E057
:102AD0009F938F938CEA93E09F938F930E94C019EA
:102AE0008DB79EB708960FB6F8949EBF0FBE8DBFE8
:102AF0000895109244028BCF809140038A3011F4E4
:102B00000C94A10D80E10E946E168111F9CF81E035
:102B10000E946E1681110C94AD0D8FEF8093BF0350
:102B20000C94DD1495980000959A000095980895EE
:102B300020E030E02817390721F000002F5F3F4FD9
:102B4000F9CF089589EB90E00C949815CF93C82F96
:102B50000E94A2159498969898B38C2F82958F70A6
:102B6000907F982B98BB0E94921598B38C2F8F70F2
:102B7000907F892B88BBCF910C949215803138F4CB
:102B8000883010F4805801C088540C94A61508951C
:102B90008091BF03803120F40E94BE158EE001C0F9
:102BA0008CE00C94A6158CE00C94A615CF93C82F3E
:102BB0000E94A215949A969898B38C2F82958F7044
:102BC000907F982B98BB0E94921598B38C2F8F7092
:102BD000907F892B88BBCF910C9492150F931F93F4
:102BE000CF93DF938C01C0E0D0E0C017D10731F064
:102BF00083E390E00E9498152196F7CFDF91CF9163
:102C00001F910F910895CF9386E990E00E94EE15F1
:102C100094989698C8B3C07FC360C8BB0E949215B1
:102C200089E290E00E94EE15C8BB0E94921581E0F7
:102C300090E00E94EE15C8BB0E94921588E20E94A7
:102C4000A61588E00E94A6158CE00E94A61581E0DA
:102C50000E94A61586E00E94A6151092BF0380E888
:102C6000CF910C94A6150F931F93CF93DF938C01F4
:102C7000C0E0D0E0C017D10731F08AE090E00E94B8
:102C8000EE152196F7CFDF91CF911F910F91089507
:102C900083B38095982F9670963011F08F7002C094
:102CA000897080619091C903891719F08093C903D5
:102CB00006C08093CB039091CA03891303C010927E
:102CC000CB0308958093CA0380EB94E09093BE03F6
:102CD0008093BD0308951092CB030895282F9091FF
:102CE000CB03982381E0921380E00895CF93DF9384
:102CF00081E00E946E16C1E0811101C0C0E088E051
:102D00000E946E16882319F0CF5FD8E001C0DC2F37
:102D100082E00E946E16882311F0CF5FD2E084E03B
:102D20000E946E16882311F0CF5FD4E0C13029F4E1
:102D300080917102D82BD0937102DF91CF910895C9
:102D4000E199FECF9FBB8EBBE09A8DB30895E199C8
:102D5000FECF9FBB8EBBE09A2DB330E0322F2227EF
:102D6000E199FECF01969FBB8EBBE09A8DB3A9017E
:102D7000480F511DCA010895AC01242F281B30E0D3
:102D80002617370788F4E199FECFF894FA013196B7
:102D90005FBB4EBBD901A453BC4F9C919DBBE29A33
:102DA000E19A7894AF01E9CF08959B01AC0161E30A
:102DB0007AE181E090E00E945219059620E030E02F
:102DC0004AE050E00E947619A4E1B0E00E94AE19FA
:102DD0000895DC01CB012FE0880F991FAA1FBB1FAC
:102DE0002A95D1F7BC01CD016B507D478A4F9F4F8B
:102DF0002AEE35E04BE050E00E947619AAE0B0E000
:102E00000E94AE190895FC01CB01A0E0B0E004C01F
:102E1000880F991FAA1FBB1F4A95D2F78083918301
:102E2000A283B3830895CF92DF92EF92FF920F9324
:102E30001F93E42FDC010D911D912D913C9113976F
:102E400068017901C60ED71EE11CF11CB701A6016D
:102E500004C03695279517950795EA95D2F7401B3C
:102E6000510B620B730B4D935D936D937C93139792
:102E70001F910F91FF90EF90DF90CF9008953F92B8
:102E80004F925F926F927F928F929F92AF92BF927A
:102E9000CF92DF92EF92FF920F931F93CF93DF9326
:102EA000E6E3F3E0C1E4D3E0ABE9B2E04EE353E0A4
:102EB00020E030E0C12CD12C76011191112361F07A
:102EC0001881111109C00D911C911197C00ED11ECE
:102ED000E11CF11C2F5F3F4F219612964E175F07A2
:102EE00061F72115310541F4809123038111C8C197
:102EF00080E180932303C4C1A90156954795C7017A
:102F0000B601640F751F811D911D40E050E00E94C5
:102F100076198091AB029091AC028217930740F42E
:102F2000281B390B3093480220934702312C08C0EC
:102F3000821B930B9093480280934702332433946F
:102F4000C0914702D0914802A0916F02B0917002E7
:102F500080906302909064026401D594C7940D2C14
:102F6000000CEE08FF089E010E9498196C0D7D1D53
:102F70008E1D9F1D092C000CAA08BB08A5019401F9
:102F80000E94761929013A018901A0912D02B09180
:102F90002E029E010E9498196C0D7D1D8E1D9F1D95
:102FA000A50194010E947619F90160914202709185
:102FB0004302C091D902D091DA0281E038120EC0EA
:102FC0004616570618F46419750902C060E070E0EF
:102FD000EC17FD07A0F4C21BD30B13C0640D751DC5
:102FE000C20FD31F8091AD0281110FC010926A02EF
:102FF00010926902109288021092870206C0C0E007
:10300000D0E0E0E0F0E000E010E080918302811188
:1030100052C0709309036093080310935A020093FF
:103020005902CB01A0E0B0E064E0880F991FAA1F0D
:10303000BB1F6A95D1F78093210290932202A0933F
:103040002302B09324029801A4E1B0E00E949819F1
:103050006093CD027093CE028093CF029093D00202
:10306000D0934602C0934502F0932A02E0932902CE
:10307000CE01A0E0B0E074E0880F991FAA1FBB1F2B
:103080007A95D1F780936B0290936C02A0936D02B6
:10309000B0936E029F01AAE0B0E00E94981960937D
:1030A000B9027093BA028093BB029093BC0281E094
:1030B00080938302E5C080910803909109032091D9
:1030C000650286179707B0F42150223060F59B0106
:1030D000281B390BE0914002F0E0EE0FFF1FE95E84
:1030E000FD4F808191812817390708F4C9C01092DB
:1030F000650219C0223099F4861B970BE0914002BB
:10310000F0E0EE0FFF1FEF5EFD4F2081318182174F
:10311000930708F4B5C081E08093650204C0681786
:103120007907C9F7ADC044E050E081E292E00E9427
:1031300013178091210290912202A0912302B09155
:10314000240224E0B695A795979587952A95D1F7FF
:103150009093090380930803209142023091430227
:103160008217930758F0821B930B90935A02809317
:10317000590210926A02109269021BC010925A0200
:1031800010925902281B390B30936A02209369026E
:103190002931310520F088E78093AD020AC0809183
:1031A000AD02882331F089E190E090936A02809328
:1031B000690244E050E0BE018BE692E00E941317E2
:1031C00080916B0290916C02A0916D02B0916E02A1
:1031D00034E0B695A795979587953A95D1F7909352
:1031E0004602809345022091D9023091DA0282177B
:1031F000930758F0821B930B90932A028093290225
:1032000010928802109287021BC010922A0210921C
:103210002902281B390B309388022093870227311B
:10322000310520F088E78093AD020AC08091AD029D
:10323000882331F087E190E09093880280938702A1
:103240002091590230915A02A4E1B0E00E949819ED
:103250006093CD027093CE028093CF029093D00200
:103260002091290230912A02AAE0B0E00E94981928
:103270006093B9027093BA028093BB029093BC0230
:10328000DF91CF911F910F91FF90EF90DF90CF9042
:10329000BF90AF909F908F907F906F905F904F9076
:1032A0003F900895DB018F939F930E94AE19BF91C9
:1032B000AF91A29F800D911DA39F900DB29F900D85
:1032C00011240895AA1BBB1B51E107C0AA1FBB1FF5
:1032D000A617B70710F0A61BB70B881F991F5A95A2
:1032E000A9F780959095BC01CD010895A1E21A2E11
:1032F000AA1BBB1BFD010DC0AA1FBB1FEE1FFF1F9A
:10330000A217B307E407F50720F0A21BB30BE40BE9
:10331000F50B661F771F881F991F1A9469F7609530
:103320007095809590959B01AC01BD01CF010895EA
:10333000A29FB001B39FC001A39F700D811D1124F6
:10334000911DB29F700D811D1124911D08950E9441
:103350009819B7FF0895821B930B08950E9498193E
:10336000A59F900DB49F900DA49F800D911D1124D9
:103370000895FB01DC0101900D920020E1F7089512
:10338000AEE0B0E0E6ECF9E10C94811C0D891E89F9
:1033900086E08C831A8309838FEF9FE79E838D835A
:1033A000AE01475E5F4F6F89788DCE0101960E9416
:1033B000E219EF81F885E00FF11F10822E96E4E00C
:1033C0000C949D1CABE0B0E0E8EEF9E10C94731CAA
:1033D0006C017B018A01FC0117821682838181FFC7
:1033E000CCC1CE0101963C01F6019381F70193FD1A
:1033F000859193FF81917F01882309F4BAC18532B9
:1034000039F493FD859193FF81917F01853229F4F1
:10341000B60190E00E94D91BE7CF912C212C312CD2
:10342000FFE1F315D8F08B3279F038F4803279F07F
:103430008332A1F4232D20611DC08D3261F08033D1
:1034400069F4232D216016C0832D8260382EE32D70
:10345000E4603E2E2AC0F32DF8601DC037FC2DC05D
:1034600020ED280F2A3040F08E32B9F436FC81C1AD
:10347000232D2064322E19C036FE06C08AE0989EA5
:10348000200D1124922E11C0EAE02E9E200D112451
:10349000222EF32DF0623F2E08C08C3621F4832DAE
:1034A0008068382E02C0883641F4F70193FD85917B
:1034B00093FF81917F018111B3CF982F9F7D955408
:1034C000933028F40C5F1F4F9FE399830DC0833620
:1034D00031F0833771F0833509F059C021C0F8010C
:1034E000808189830E5F1F4F88248394912C530120
:1034F00013C02801F2E04F0E511CF801A080B180EA
:1035000036FE03C0692D70E002C06FEF7FEFC5018A
:103510000E94CE1B4C018201F32DFF773F2E16C077
:10352000280122E0420E511CF801A080B18036FE35
:1035300003C0692D70E002C06FEF7FEFC5010E94EC
:10354000C31B4C01F32DF0683F2E820133FC1BC0DE
:10355000822D90E088169906B0F4B60180E290E0E2
:103560000E94D91B2A94F4CFF50137FC859137FED0
:1035700081915F01B60190E00E94D91B21102A942D
:1035800021E0821A91088114910471F7E8C0843611
:1035900011F0893641F5F80137FE07C0608171816D
:1035A000828193810C5F1F4F08C060817181072E5B
:1035B000000C880B990B0E5F1F4FF32DFF763F2EEB
:1035C00097FF09C090958095709561957F4F8F4FBB
:1035D0009F4FF0683F2E2AE030E0A3010E94151CA7
:1035E000882E861845C0853731F4232D2F7EB22EC4
:1035F0002AE030E025C0932D997FB92E8F36C1F097
:1036000018F4883579F0B5C0803719F0883721F083
:10361000B0C0E92FE061BE2EB4FE0DC0FB2DF460FA
:10362000BF2E09C034FE0AC0292F2660B22E06C064
:1036300028E030E005C020E130E002C020E132E0C7
:10364000F801B7FE07C060817181828193810C5FB0
:103650001F4F06C06081718180E090E00E5F1F4FB8
:10366000A3010E94151C882E8618FB2DFF773F2E84
:1036700036FE0DC0232D2E7FA22E891458F434FE61
:103680000BC032FC09C0832D8E7EA82E05C0B82C3D
:10369000A32C03C0B82C01C0B92CA4FE0FC0FE019E
:1036A000E80DF11D8081803321F49A2D997EA92E99
:1036B00009C0A2FE06C0B394B39404C08A2D8678D4
:1036C00009F0B394A3FC11C0A0FE06C0B21488F4A4
:1036D000280C922C9B180EC0B21460F4B60180E244
:1036E00090E00E94D91BB394F7CFB21418F42B18B2
:1036F00002C0982C212CA4FE10C0B60180E390E0FB
:103700000E94D91BA2FE17C0A1FC03C088E790E06D
:1037100002C088E590E0B6010CC08A2D867859F089
:10372000A1FE02C08BE201C080E2A7FC8DE2B601DF
:1037300090E00E94D91B891438F4B60180E390E030
:103740000E94D91B9A94F7CF8A94F301E80DF11DDA
:103750008081B60190E00E94D91B8110F5CF222014
:1037600009F442CEB60180E290E00E94D91B2A946F
:10377000F6CFF6018681978102C08FEF9FEF2B96DF
:10378000E2E10C948F1CFC01059061507040011027
:10379000D8F7809590958E0F9F1F0895FC0161507A
:1037A000704001900110D8F7809590958E0F9F1F63
:1037B00008950F931F93CF93DF93FB01238121FD86
:1037C00003C08FEF9FEF2CC022FF16C046815781A8
:1037D000248135814217530744F4A081B1819D01B2
:1037E0002F5F3F4F318320838C93268137812F5F5A
:1037F0003F4F3783268314C08B01EC01FB0100840B
:10380000F185E02D0995892BE1F6D80116968D9169
:103810009C911797019617969C938E931697CE01BD
:10382000DF91CF911F910F910895FA01AA272830B7
:1038300051F1203181F1E8946F936E7F6E5F7F4F7D
:103840008F4F9F4FAF4FB1E03ED0B4E03CD0670FF9
:10385000781F891F9A1FA11D680F791F8A1F911D4C
:10386000A11D6A0F711D811D911DA11D20D009F49C
:1038700068943F912AE0269F11243019305D3193DE
:10388000DEF6CF010895462F4770405D4193B3E0C7
:103890000FD0C9F7F6CF462F4F70405D4A3318F06E
:1038A000495D31FD4052419302D0A9F7EACFB4E01F
:1038B000A6959795879577956795BA95C9F70097D7
:1038C0006105710508959B01AC010A2E0694579578
:1038D000479537952795BA95C9F7620F731F841FCF
:1038E000951FA01D08952F923F924F925F926F9265
:1038F0007F928F929F92AF92BF92CF92DF92EF9280
:10390000FF920F931F93CF93DF93CDB7DEB7CA1B00
:10391000DB0B0FB6F894DEBF0FBECDBF09942A882B
:10392000398848885F846E847D848C849B84AA84D3
:10393000B984C884DF80EE80FD800C811B81AA8160
:10394000B981CE0FD11D0FB6F894DEBF0FBECDBF2B
:08395000ED010895F894FFCF8A
:10395800526573756C7473205265706F7274656408
:1039680000202056657273696F6E2025752E2530EC
:1039780032752020002020436F6E66696775726972
:103988006E67202020002020496E697469616C6987
:103998007A696E67202000556E6974733A2020207A
:1039A80020202020202020004C6F61642043656C7B
:1039B8006C733A202020204B004C43207820456E21
:1039C80061626C653A202020200052652D496E699D
:1039D800742042696E3A2020202000456D70747969
:1039E8002042696E3A202530356C75004E756D2081
:1039F8004C6567733A2020202020202530316C75D3
:103A08000049443A20202020202020202530356CF1
:103A1800750046756C6C42696E206C623A253035CB
:103A28006C750046756C6C42696E206B673A253080
:103A3800356C750046756C6C42696E3A446F20456A
:103A48006D7074790046756C6C42696E3A4E6F20E1
:103A580043656C6C730046756C6C42696E3A4164E0
:103A68006420466565640046756C6C42696E3A2050
:103A78004F4F522020202000456D747942696E20F6
:103A88006C623A2530356C7500456D747942696E03
:103A9800206B673A2530356C75005765696768741F
:103AA80020746F6F206C61726765004C432045720B
:103AB800726F72202020202020202575005065720A
:103AC800666F726D3A2020456D70747920005265DA
:103AD8002D706572666F726D20456D707479005730
:103AE8006569676874206C62733A2530356C7500B7
:103AF800576569676874206B673A202530356C759F
:0E3B08000003000400050005000A000F000085
:00000001FF
